S02B000062696E2F6F70656E626C745F64656D6F70726F675F6E75636C656F5F73746D33326631303372622EC3
S31508000000F0060020FD0F0008E10F0008E10F0008C8
S31508000010E10F0008E10F0008E10F0008E10F0008F2
S31508000020E10F0008E10F0008E10F0008E10F0008E2
S31508000030E10F0008E10F0008E10F0008E10F0008D2
S31508000040E10F0008E10F0008E10F0008E10F0008C2
S31508000050E10F0008E10F0008E10F0008E10F0008B2
S31508000060E10F0008E10F0008E10F0008E10F0008A2
S31508000070E10F0008E10F0008E10F0008E10F000892
S31508000080E10F0008E10F0008E10F0008E10F000882
S31508000090E10F0008E10F0008E10F0008E10F000872
S315080000A0E10F0008E10F0008E10F0008E10F000862
S315080000B0E10F0008E10F0008E10F0008E10F000852
S315080000C0E10F0008E10F0008E10F0008E10F000842
S315080000D0E10F0008E10F0008E10F0008E10F000832
S315080000E0E10F0008E10F0008E10F0008E10F000822
S315080000F0E10F0008E10F0008E10F0008E10F000812
S31508000100E10F0008E10F0008E10F0008E10F000801
S31508000110E10F0008E10F0008E10F0008E10F0008F1
S31508000120E10F0008E10F0008E10F0008E10F0008E1
S31508000130E10F0008E10F0008E10F0008E10F0008D1
S31508000140E10F0008E10F0008E10F0008E10F0008C1
S3150800015000B583B00023009301934FF48053C4F293
S3150800016002031A6842F001021A6059680022CFF6A3
S31508000170FF020A405A601A6822F0847222F480321A
S315080001801A601A6822F480221A605A6822F4FE025B
S315080001905A604FF41F029A601A6842F480321A6055
S315080001A04FF48053C4F2020340F2DC52196801F49A
S315080001B000310191009901310091019911B9009915
S315080001C09142F3D14FF48053C4F202031B6813F42F
S315080001D0003F06D141F26000C0F600006E2100F033
S315080001E0FFFA4FF40053C4F202031A6842F01002F1
S315080001F01A601A6822F003021A601A6842F00202AC
S315080002001A604FF48053C4F202035A685A605A6857
S3150800021042F400525A605A6842F480625A605A6838
S3150800022022F47C125A605A6842F4E8125A601A6834
S3150800023042F080721A604FF48053C4F202031A68BF
S3150800024012F0007FFBD04FF48053C4F202035A68C1
S3150800025022F003025A605A6842F002025A604FF4CA
S315080002608053C4F202035A6802F00C02082AFAD133
S315080002704FF48053C4F20203DA6942F40032DA61B9
S315080002809A6942F005029A614FF40063C4F20103C9
S315080002901A6822F470621A601A6842F430621A60A8
S315080002A01A6822F470421A601A6842F480421A6088
S315080002B000F004F800F010F8FCE700BF08B500F0FD
S315080002C093FA00F089FA00F0C9FB00F0A9FB00F0E8
S315080002D00DF800F06FFA08BD08B500F07FFA00F0D7
S315080002E0D9FB00F00FF800F045FA08BD08B500F094
S315080002F063F800F0CFFA40F20003C2F200030022CE
S315080003001A7008BD08B540F20400C2F2000000F0F9
S315080003100BFB01280BD140F20003C2F200030022B6
S315080003201A7040F20400C2F2000000F065F808BD39
S31508000330704700BF08B540F20003C2F200031B78FD
S3150800034013B9C9B200F0BCFA00F04EF808BD00BFF8
S3150800035040F20003C2F200031878022806D00328E8
S3150800036006D001280CBF082040207047002070479F
S315080003700020704740F20003C2F2000318780228F2
S3150800038006D0032806D001280CBF08204020704755
S31508000390002070470020704708B500F01BF808BD1C
S315080003A040F24403C2F20003FE22DA7018710222F8
S315080003B0A3F84420704700BF40F24403C2F200038A
S315080003C000221A709A6483F84320A3F844209A708E
S315080003D05A70704740F24403C2F20003187800309E
S315080003E018BF0120704700BF40F24403C2F2000361
S315080003F0002283F84320704738B504460178FF2960
S315080004001ED140F24404C2F20004002363700125A1
S315080004102570FF22E270102222716371FFF798FFA0
S31508000420A071FFF7A7FFE071FFF7A4FF000A20728B
S315080004306572A5720823A4F8443000F0F1FA79E150
S3150800044040F24403C2F200031B78012B40F090816E
S31508000450C939352900F26B81DFE811F0DB00690143
S3150800046069016501690169015901FC0042012F0111
S31508000470690169016901690169016901690169011E
S31508000480690169016901690169016901690169010E
S3150800049069016901690169016901690169016901FE
S315080004A069016901690169016901690169016901EE
S315080004B07F00540036007300690169016901A100D3
S315080004C06901B900BD00CE004578FFF741FF013844
S315080004D0854203DD2220FFF763FF2BE140F2440546
S315080004E0C2F20005281DA96C627800F09BF9FF236B
S315080004F0EB706278AB6C1344AB6463780133A5F890
S31508000500443017E14578FFF723FF0138854203DDBC
S315080005102220FFF745FF0DE1616840F24405C2F26B
S315080005200005A964281D627800F07CF9FF23EB70AA
S315080005306278AB6C1344AB6463780133A5F8443036
S31508000540F8E040F24403C2F20003FF22DA70426880
S315080005509A640122A3F84420ECE040F24403C2F274
S315080005600003FF22DA709B6C406840B118440022F1
S3150800057013F8011B0A44D2B28342F9D100E00022E3
S3150800058040F24403C2F20003C3F8072001221A719D
S3150800059000225A719A710822A3F84420CAE040F250
S315080005A04403C2F20003FF22DA7041F26802C0F681
S315080005B000029A6400221A715A719A710721D97138
S315080005C01A725A729A720822A3F84420B2E00020DE
S315080005D0FFF7E6FEAEE040F24403C2F20003FF2254
S315080005E0DA7000221A71597859719A71DA711A7289
S315080005F00622A3F844209DE040F24403C2F2000319
S3150800060000221A705A70FF22DA700122A3F84420D9
S3150800061090E040F24403C2F200039D6CFFF798FE97
S31508000620411E2846621C00F0FFF918B93120FFF771
S31508000630B7FE7FE040F24404C2F20004FF23E370F1
S31508000640A56CFFF785FE013D2844A0640123A4F8A4
S3150800065044306FE04578FFF77BFE0238854203DDBC
S315080006602220FFF79DFE65E040F24403C2F2000334
S31508000670FF22DA700122A3F84420617839B900F024
S31508000680E3F9002856D13120FFF78AFE52E040F2FE
S315080006904403C2F20003986CA21C00F0C5F918B90D
S315080006A03120FFF77DFE45E040F24403C2F2000325
S315080006B061789A6C0A449A643CE040F24404C2F2B7
S315080006C00004FF23E370002525716571FFF740FEDE
S315080006D0A071E571257265720723A4F8443029E0F4
S315080006E040F24403C2F20003986C616800F0A0F976
S315080006F018B93120FFF754FE1CE040F24403C2F259
S315080007000003FF22DA700122A3F8442012E000F069
S315080007106FF840F24403C2F20003FF22DA700122A6
S31508000720A3F8442006E03120FFF73AFE02E0202035
S31508000730FFF736FE40F24403C2F2000393F8433053
S31508000740012B02D11020FFF72BFE40F24403C2F220
S315080007500003B3F844100BB2002B09DD40F2440045
S31508000760C2F20000012380F843300330FFF7E2FDB0
S3150800077038BD00BF08B5FFF70FFE012819D040F2B3
S315080007809003C2F200031B78012B12D100F094F9F2
S3150800079040F29403C2F200031B6803F5FA73984209
S315080007A007D340F29003C2F2000300221A7000F049
S315080007B01FF808BD08B540F29003C2F200030122F3
S315080007C01A7000F079F940F29403C2F20003186037
S315080007D0FFF7D0FF08BD00BF704700BF704700BFD6
S315080007E008B5FFF7FBFFFCE708B500F003FC08BDFA
S315080007F010B500F021F9A0B1FFF79AFD00F042F913
S3150800080000F01EF920F0604020F07F004EF60853F5
S31508000810CEF20003186000F013F9446800F0ECFB10
S31508000820A04710BD70B5561EB6B24AB14C1E0E444E
S31508000830451A14F8013F2B55FFF7D0FFB442F8D1FB
S3150800084070BD00BF10B54FF48843C4F200031B887F
S3150800085003F080039BB2B3B14FF48843C4F200039C
S3150800086098801B8803F080039BB273B94FF48844C1
S31508000870C4F20004FFF7B2FF238803F080039BB29B
S31508000880002BF7D003E0002010BD012010BD012089
S3150800089010BD00BF4FF48843C4F2000300221A813A
S315080008A09A811A829A821A8340F271221A819A8947
S315080008B092B242F4005242F00C029A81704700BF8D
S315080008C02DE9F04106460C46402906D941F270004A
S315080008D0C0F600008D21FFF783FF2046FFF7B2FF21
S315080008E0012806D041F27000C0F600009121FFF7FA
S315080008F077FF2546ACB1002441F27007C0F6000721
S315080009004FF09A08FFF76AFF305DFFF79BFF012853
S3150800091003D038464146FFF763FF0134A3B2AB4222
S31508000920F0D3BDE8F08100BF10B540F2E103C2F292
S3150800093000031B785BBB4FF48843C4F200031B8893
S3150800094003F020039BB2002B56D04FF48843C4F221
S3150800095000039A8892B240F29C03C2F200031A700E
S3150800096012F0FF0F4AD000F0A7F840F29803C2F23F
S315080009700003186040F2E003C2F20003002018707A
S3150800098040F2E103C2F2000301221A7010BD40F2E0
S31508000990E003C2F200031A784FF48843C4F2000356
S315080009A01B8803F020039BB263B34FF48843C4F259
S315080009B000039C8840F29C03C2F2000399184C700D
S315080009C00132D2B240F2E001C2F200010A701B788D
S315080009D0934215D11149FFF725FF40F2E103C2F210
S315080009E0000300221A70012010BD40F2E103C2F292
S315080009F000030020187010BD002010BD002010BD97
S31508000A00002010BD00F058F840F29803C2F2000327
S31508000A101B6864339842E8D8002010BD9D0000206A
S31508000A2008B500F05BF908BD08B500F065F908BD22
S31508000A3008B500F089F908BD08B500F071FA08BDD7
S31508000A4008B500F0C7FA08BD08B500F03DFA10B1C0
S31508000A5000F09AFA08BD002008BD00BF4EF2100348
S31508000A60CEF2000300221A6041F63F11C0F20101DE
S31508000A7059609A600521196040F2E403C2F2000346
S31508000A801A6070474EF21003CEF2000300221A6075
S31508000A90704700BF4EF21003CEF200031B6813F432
S31508000AA0803F1FBF40F2E403C2F200031A68013216
S31508000AB018BF1A60704700BF08B5FFF7EBFF40F292
S31508000AC0E403C2F20003186808BD00BF4FF40053E0
S31508000AD0C4F202031A6942F080021A61704700BF25
S31508000AE0F8B507460024254641F29806C0F60006E2
S31508000AF0FFF774FEA359BB420ED8311949680B4457
S31508000B009F4209D241F29803C0F6000305EB45025D
S31508000B1003EB8203187AF8BD01350C349C2CE7D117
S31508000B20FF20F8BD2DE9F84380460068FFF7D8FF97
S31508000B30FF285CD04FF40053C4F2020340F223129C
S31508000B40C4F267525A6048F6AB12CCF6EF525A60B6
S31508000B503422DA60DB6813F0010F04D0FFF7B6FF22
S31508000B600020BDE8F8834FF40053C4F202031A6963
S31508000B7042F001021A61002508F104094FF40054F5
S31508000B80C4F20204D8F80030EF1859F80560B2B27A
S31508000B90EA52E36813F0010F05D0FFF71FFEE3687A
S31508000BA013F0010FF9D1330C7B80E36813F0010FC2
S31508000BB005D0FFF713FEE36813F0010FF9D13B6880
S31508000BC0B34204D10435B5F5007FDBD101E000243A
S31508000BD000E001244FF40053C4F202031A6922F01C
S31508000BE001021A61FFF772FF2046BDE8F88300206C
S31508000BF0BDE8F88338B504460D4640F2E803C2F26C
S31508000C000003984209D04FF4C043C0F60003994246
S31508000C100BD0FFF787FF20B917E040F2EC24C2F2A9
S31508000C200004C5F3080393B903E040F2E804C2F2EE
S31508000C30000423689D420CD0204640F8045B2946F0
S31508000C404FF40072FFF7EEFD03E0002038BD0020E8
S31508000C5038BD204638BD00BF2DE9F04106460C4692
S31508000C6017461D464FEA51284FEA48280368B3F14C
S31508000C70FF3F06D140F8048B41464FF40072FFF758
S31508000C80D1FD3368434505D030464146FFF7B2FFEC
S31508000C900646D0B13368E41A3444043408F50078BB
S31508000CA0FFF79CFD331DE31AB3F5007F06D33046E4
S31508000CB04146FFF79FFF064650B1041D17F8013B52
S31508000CC004F8013B013DEBD105E00020BDE8F081C9
S31508000CD00020BDE8F0810120BDE8F08140F2EC2358
S31508000CE0C2F200034FF0FF321A6040F2E803C2F284
S31508000CF000031A60704700BF70B504460D461646D5
S31508000D00FFF7EEFEFF281BD0681E2044FFF7E8FE1B
S31508000D10FF2817D0620A4FF4C043C0F60003B3EBAE
S31508000D20422F07BF40F2E800C2F2000040F2EC2072
S31508000D30C2F20000214632462B46FFF78DFF70BDF2
S31508000D40002070BD002070BD2DE9F84304460E460C
S31508000D50FFF7C6FE0546701E2044FFF7C1FE04468F
S31508000D60FF2D18BFFF2800F0AB80854200F29F8058
S31508000D70022D40F29F800F2800F29F804FF4005307
S31508000D80C4F2020340F22312C4F267525A6048F6CC
S31508000D90AB12CCF6EF525A603422DA60DB6813F0F5
S31508000DA0010F04D0FFF792FE0020BDE8F8834FF448
S31508000DB00053C4F202031A6942F002021A6141F2B0
S31508000DC09809C0F600094F460026FFF707FD3B7A4B
S31508000DD0AB4208D141F29803C0F6000306EB46027F
S31508000DE053F8227005E001360C370D2EEDD14FF081
S31508000DF0FF37C8460025FFF7F1FC98F80830A342EC
S31508000E0008D141F29803C0F6000305EB450253F8F2
S31508000E10228006E0013508F10C080D2DEBD14FF0C4
S31508000E20FF384E460025FFF7D9FC337AA34209D18D
S31508000E3041F29803C0F6000305EB450203EB820373
S31508000E405B6804E001350C360D2DECD10023C7EBA9
S31508000E5008084344C3F38F23E3B1013B9EB201362E
S31508000E60B60200254FF40054C4F20204EB1963617C
S31508000E70236943F040032361E36813F0010F05D0AB
S31508000E80FFF7ACFCE36813F0010FF9D105F58065AF
S31508000E90B542EBD14FF40053C4F202031A6922F0AB
S31508000EA002021A61FFF712FE0120BDE8F88300204E
S31508000EB0BDE8F8830020BDE8F8830020BDE8F88384
S31508000EC00020BDE8F88300BF00B583B040F2E80310
S31508000ED0C2F200031B68B3F1FF3F08BF01201CD014
S31508000EE040F2E803C2F2000399685A681144DA68C6
S31508000EF011441A6911445A6911449A690A44D9690C
S31508000F0053185B4202AA42F8043D46F25010C0F656
S31508000F1000000421FFF7F0FEFFE703B05DF804FBCD
S31508000F2046F20402C0F600024FF4C043C0F60003BE
S31508000F3010681B68184446F20803C0F600031B68CD
S31508000F40184446F20C03C0F600031B68184446F220
S31508000F501003C0F600031B68184446F21403C0F6D3
S31508000F6000031B68184446F21803C0F600031B6802
S31508000F70184446F25013C0F600031B681844D0F113
S31508000F80010038BF0020704708B540F2E803C2F2F6
S31508000F9000031B68B3F1FF3F06D040F2E800C2F237
S31508000FA00000FFF7BFFD88B140F2EC23C2F2000350
S31508000FB01B68B3F1FF3F0BD040F2EC20C2F20000F1
S31508000FC0FFF7B0FD003018BF012008BD002008BD9E
S31508000FD0012008BD4FF4C040C0F60000704700BFAE
S31508000FE008B541F23410C0F600003121FFF7F8FBCE
S31508000FF008BD00BF72B6704762B6704710B515498E
S315080010008D4640F20002C2F2000240F20103C2F22B
S3150800101000039A4210D2131D0D4CE41A24F003045F
S3150800102004340023104641F26411C0F600015A58F0
S315080010301A500433A342FAD1074808494FF0000270
S315080010408842B8BF40F8042BFADBFFF781F810BDD9
S3150800105004000020F006002004000020F004002010
S315080010606D61696E2E6300004F70656E424C5400C8
S315080010702E2E2F2E2E2F2E2E2F536F757263652F21
S3150800108041524D434D335F53544D333246312F75DC
S315080010906172742E630000000060000800200000E2
S315080010A00300000000800008002000000400000083
S315080010B000A00008002000000500000000C000088D
S315080010C0002000000600000000E0000800200000E4
S315080010D007000000000001080020000008000000CA
S315080010E00020010800200000090000000040010857
S315080010F0002000000A00000000600108002000002F
S315080011000B00000000800108002000000C00000011
S3150800111000A00108002000000D00000000C0010822
S31508001120002000000E00000000E00108002000007A
S315080011300F0000002E2E2F2E2E2F2E2E2F536F75BA
S315080011407263652F41524D434D335F53544D3332CD
S3150800115046312F4743432F766563746F72732E6348
S30908001160000000007D
S306080011640478
S70508000000F2
